:020000040000FA
:0400000006EF00F017
:0800080050EF02F0C26ACD8046
:10001000060EC16E9D902C0E926EFF0E936E946E26
:10002000956E966AF18E120E806EF28CF28E0E6ACA
:1000300083AE0E802CDA8092050E026E959C070E20
:10004000846E05DA060E846E02DA839C00DA838CF5
:10005000022EF5D7958C000E846E05D809B014D801
:1000600080A49DD8FAD7099080BA0DD0ECD9100E93
:10007000026EEBD901360036018080AA0190022E73
:10008000F8D7E3D909801200080E046E000E056E41
:1000900076D8005CD8B402D0040E05D070D8015CCC
:1000A000D8B41AD0030E036E70D8032EFDD70450B7
:1000B0001108D8A008D0D8A4EBD705508808D8A03C
:1000C00002D0D8A4E5D70D8040D8060E846EBFD9E3
:1000D0008082D7D90B9025D052D80C6E50D8066E9E
:1000E0004ED8076E0D9031D80650046E0750056E3D
:1000F00046D8026E02AC08D0040E026EBCD91E0EA9
:1001000096D9022EFBD7DFD7010E02BE030E026E78
:10011000070E846E80929BD98082A7D9022EFAD7CF
:100120000B80000E846E80920EA00ED0808297D934
:1001300000381AD892D9005017D88FD9013814D85E
:100140008CD9015011D880921200929A809A320E66
:100150000DB0050E6CD9808A928A0DA002D02D0EAA
:1001600066D9190E64D912000F0B026ED8A402D002
:1001700088D904D080D96DD9022EFCD712000AD8B4
:10018000086EF95002D808501200020E0526D8B4A5
:10019000042A1200FB6A0450FA6E0550F96E030E31
:1001A0000CB8010E0EB0010E106E1C6A0D6A0650DE
:1001B000046E0750056EACD814BEB4D8E0DF186EDC
:1001C000C1D81150846E31D90D901C6A1D6A010E80
:1001D0001E6EAFD81BAC2DD0D2DF1C6E0CAA02D085
:1001E0001C961C981CB021D01CB217D01CB40DD08A
:1001F0001CB61FD01CB866D01CBA03D01CBC15D0CE
:100200003FD0800E0CBA1B1214D01950126E1A5027
:10021000136E1B50146E96D833D01950156E1A50A9
:10022000166E1B503F0B176E2BD0A9DF1D6EA7DF7C
:100230001E6E91D81BAE0CD01CAC96D81CBCA3D89B
:10024000010E1E5ED8A01D5E1D501E10D8A4F4D74E
:1002500019500CBCFF0A81181214D8A40FD01A50E0
:100260000CBCFF0A82181314D8A408D01B500CBC75
:10027000FF0A831814143F0BD8B402D00D800D82EE
:100280009CD80FB027D0C9D8182E9ED70CAE22D03C
:1002900076DF186E0D904DD85ED8A4D880B6FED704
:1002A000195081181214D8A40BD01A5082181314A4
:1002B000D8A406D01B50831814143F0BD8B402D016
:1002C0000D800D827AD80FB005D0A7D880A6FED7B2
:1002D000182EE0D7FF0E936E946E956E102E67D792
:1002E0000D420EB002D0B1D830DF0DB003D0BDD872
:1002F000070E02D0C6D8060E846E0A0E026EA7D86C
:100300008082A5D88092022EFAD7000E846E120049
:1003100036DF116E119E33DF126E31DF136E2FDF69
:10032000146E12002CDF156E2ADF166E28DF176E92
:10033000120025DF196E23DF1A6E21DF1CB8800939
:100340001B6E12001250936E1350946E14503F0B9C
:10035000C009956E12001950816E1A50826E1B50A2
:100360003F0B836E5AD812001550811A1650821A0C
:100370001750831A52D81550811A1650821A1750E6
:10038000831A4BD81200800E1F6E206A1550811AF6
:100390001650821A1750831A000000001550811A57
:1003A0001650821A1750831A010E205ED8A01F5EC5
:1003B0001F502010D8A4EAD712000F900EA011D021
:1003C000C4DE0DB002D051D801D05BD8959C839C7F
:1003D00083AE04D080B4FCD70F800D82838C958CC3
:1003E0003AD81200809831D814501BBE800907D823
:1003F000135005D8125003D8808827D812000A6EEF
:10040000080E026E0A36D8B002D0809802D08088DA
:1004100000001BD8022EF6D71200050E216E000038
:1004200000000000212EFDD712003B0EF7D7236EEF
:100430000A0E226E00D000D00000F7DF222EFCD77B
:10044000232EF6D71200020EF2D7040EF0D7640E58
:10045000EED7C80EECD7FA0EEAD7F9DFFAD70A0EB4
:10046000246EF5DF242EFDD71200F60E256EAB0E9E
:10047000266E640E11D0F30E256E8B0E266E640E62
:100480000BD0ED0E256E560E266EFA0E05D0F3DF5C
:100490001E0ECDDFEADF12009D80C9DF9D901200A5
:1004A000276ED8CF28F0E0CF29F09EA006EF00F00D
:1004B0002550CF6E2650CE6E010E801A9E9029C018
:1004C000E0FF275028C0D8FF1000436F7079726991
:1004D0006768742028432920323031302D32303182
:1004E00038206279204D2E59616D616D6F746F00F7
:10080000000C000C000C180C000C000C010C800CEF
:10081000180C220C000C020C000C180C580C000CCC
:10082000030C800C180C7A0C000C040C000C180C37
:10083000B00C000C050C800C180CC60C000C060C3F
:10084000800C180CC60C000C070C800C180CE40C67
:10085000000C080C000C190C020C000C090CA00C6C
:10086000190C020C000C100C000C190C340C000CB0
:10087000110C400C190C340C000C140C000C180C4E
:10088000B00C000C160C800C180CC60C000C170CCD
:10089000800C180CE40C000C200C000C190C6E0CD5
:1008A000000C210C400C190C6E0C000C270C000CD9
:1008B000190CD80C000C300C000C1A0C120C000C8B
:1008C000320C000C1A0C580C000C370C000C180CD5
:1008D000000C000C380C800C180C7A0C000C400C2E
:1008E000000C190C6E0C000C420C000C1A0C7A0C4B
:1008F000000C460C100C1A0CE40C000C470C100CED
:100900001A0CE40C000C480C600C1A0CE40C000CE3
:10091000510C000C1B0C680C100C510C000C1B0C27
:10092000B40C000C720C000C1B0CE80C000C730CCB
:10093000000C1C0C2E0C100C730C000C1C0C680C06
:10094000900C730C000C1C0CA20C000C740C000C12
:100950001C0CDC0C000C750C000C1D0C160C900C07
:10096000750C000C1D0C380C000C760C000C1D0CCA
:100970005A0C900C760C000C1D0CA00C000C770C83
:10098000000C1D0CE60C900C770C000C1E0C080CD7
:10099000000C780C000C1E0C2A0C900C780C000C2F
:1009A0001E0C700C000C830C000C1E0CB60C900C72
:1009B000830C000C1E0CC60C000C850C000C1E0CCD
:1009C000D60C000C860C000C1F0C320C000C900C8A
:1009D000000C1F0C540C900C900C000C1F0CAC0C59
:1009E000000C910C000C1F0CBC0C900C910C000C1A
:1009F000200C020C000C920C000C200C480C900CEB
:100A0000920C000C200CA00C000C930C000C200C81
:100A1000B00C900C930C000C210C200C000C950CCD
:100A2000000C210C300C000C960C000C210C6C0CF2
:100A3000900C960C000C210CD00C010C070C000C37
:100A4000220C340C110C070C000C220C6E0C010C47
:100A5000080C000C220CA80C010C090C000C220C38
:100A6000EE0C010C120C000C230C340C010C130CBA
:100A7000000C230C7A0C010C250C800C230CB40CFC
:100A8000010C260C800C230CD80C010C310C000C32
:100A9000230CFC0C010C320C000C180C000C010C8B
:100AA000330C000C240C4E0C010C370C000C240CE5
:100AB000AC0C010C380C000C240CF80C010C390C9B
:100AC000000C250C440C010C410C100C250C6C0C7A
:100AD000910C410C100C250CDE0C010C470C000C89
:100AE000260C500C010C480C000C260C960C010C2A
:100AF000490C000C260CDC0C010C510C000C270CD2
:100B0000220C010C520C000C270C920C010C530C03
:100B1000000C270CFC0C010C540C000C280C4C0C89
:100B2000010C550C000C280CC80C010C570C000CC7
:100B3000280CF60C010C580C400C280CF60C010C7F
:100B4000600C000C290C1E0C010C610C000C290C13
:100B50006C0C010C620C200C290C1E0C010C630C9B
:100B6000200C290C6C0C010C640C000C290CBA0C28
:100B7000010C650C000C2A0C1E0C010C660C000C00
:100B80002A0C700C010C730C800C2A0CD40C010C78
:100B9000740C000C2B0C1C0C010C750C000C2B0C99
:100BA0004A0C010C820C000C2B0C840C010C900CD8
:100BB000000C2B0C8E0C010C910C000C2C0C1C0C42
:100BC000010C920C000C2C0CAA0C010C930C000CC8
:100BD0002D0C1C0C010C940C000C2D0C9E0C010C0B
:100BE000950C000C2E0C140C020C370C400C240C31
:100BF000AC0C020C380C400C240CF80C020C400C11
:100C0000800C2E0C660C020C410C800C2E0C8A0CF5
:100C1000020C420C800C2E0CAE0C020C430CC00CCF
:100C20002E0CAE0C020C440CC00C2E0C660C020CEC
:100C3000450C800C2E0CFA0C020C460C000C2F0CF0
:100C40003A0C020C470C100C2F0C3A0C020C480CFE
:100C5000600C2F0C3A0C020C490C400C2F0C3A0C77
:100C6000020C510C800C2F0CBE0C020C530CA00C6F
:100C7000270CFC0C020C570C800C300C060C020CE0
:100C8000580CC00C300C060C020C590C000C300C2B
:100C9000360C020C660C800C300CB20C020C730C7F
:100CA000000C300CE20C020C790C000C310C0A0C1C
:100CB000020C800C000C310C2C0C020C830C000C70
:100CC000310C720C020C920C100C310C820C020CC8
:100CD000940C100C310C980C020C980C000C320C7B
:100CE000440C020C990C800C320C600C030C230C8D
:100CF000800C320CBA0C030C520C800C330C140C0C
:100D0000030C530CA00C330C140C030C540C800C6F
:100D1000330C640C030C560C800C330CF40C030CD9
:100D2000650C800C340C8A0C030C660CC00C340C63
:100D30008A0C030C670C800C340CBA0C030C680C86
:100D4000C00C340CBA0C030C730C800C340CDE0C8D
:100D5000030C740C800C350C0E0C030C750C000C81
:100D6000350C440C030C770C000C350C660C030C92
:100D7000780C000C350C8E0C030C790C000C350C27
:100D8000B60C030C860C000C350CDE0C030C900C1E
:100D9000000C360C000C130C900C000C360C340CB0
:100DA000030C930C000C360C860C040C420C000C4B
:100DB000360CD20C040C430C000C360CDC0C040C6E
:100DC000440C000C360CE60C040C900C000C360C99
:100DD000F00C050C330CC00C340CDE0C050C340C80
:100DE000C00C350C0E0C050C400C800C370C480C5C
:100DF000050C410CC00C370C480C050C630C800C26
:100E0000370C780C050C640C800C370CB40C050CFA
:100E1000730CC00C370C780C050C740CC00C370C20
:100E2000B40C050C900C800C370CEA0C050C920CE1
:100E3000000C380C7C0C050C950C800C380CFE0C4E
:100E4000050C970C000C390C0E0C060C200C800CB9
:100E5000390C1E0C060C230CC00C390C1E0C060C95
:100E6000400CC00C2E0CFA0C060C430C800C390CF8
:100E7000520C060C460C000C390C920C060C520C51
:100E8000000C390C9C0C060C680C000C390CA60CE0
:100E9000060C690C000C3A0C040C060C700C000CCF
:100EA0003A0C620C060C790C000C3A0C6C0C060C1B
:100EB000800C000C3A0C760C060C820C000C3A0CE0
:100EC000800C060C840C000C3A0C8A0C060C880C66
:100ED000000C3A0C940C060C970C000C3A0C9E0C6F
:100EE000400C000C000C3A0CA80C400C010C000C3F
:100EF0003A0CD00C400C020C000C3A0CF20C400CDA
:100F0000070C000C3B0C200C400C110C000C3B0C93
:100F1000420C400C120C000C3B0C640C400C130CEB
:100F2000000C3B0C920C400C140C200C3E0C3A0CA8
:100F3000400C150C000C3B0CC00C400C160C800C2B
:100F40003B0CF40C400C170C000C3C0C180C400C27
:100F5000180C000C3C0C900C400C190C000C3D0CB7
:100F60002A0C400C200C100C3D0C880C400C210C61
:100F7000000C3E0C3A0C400C220C000C3E0C8E0C6B
:100F8000400C230C000C3E0CE00C400C240C000C1C
:100F90003F0C080C400C250C000C3F0C840C400C42
:100FA000270C000C3F0CAC0C400C280C000C3F0C28
:100FB000F20C400C290C000C400C5C0C400C300C6A
:100FC000000C400CF60C400C400C100C410C180CA2
:100FD000400C430C800C410CC40C400C440C800CA5
:100FE000410CFA0C400C450C100C420C300C400C1F
:100FF000490C000C420C460C900C490C000C420CA5
:101000005C0C400C500C400C420C460C900C500CEC
:10101000400C420C5C0C400C510C000C420C720C4D
:10102000400C520C000C420CE80C400C530C000C11
:10103000430C2E0C400C600C100C430C740C400C38
:10104000630C200C1E0CD60C400C660C800C3B0C68
:10105000F40C400C680C000C440C140C400C690C93
:10106000000C440C5A0C400C700C000C400CF60C9C
:10107000400C710C400C3A0CD00C400C720C400C23
:101080003A0CF20C400C730C400C3E0CE00C400C83
:10109000750C400C3F0C840C400C760C800C440CFE
:1010A000700C400C770C400C400CF60C400C780C8B
:1010B000000C440CB80C400C810C400C3B0C420C56
:1010C000400C820C400C3B0C640C400C860C000C59
:1010D000440CFE0C400C930C000C3B0C420C400CDE
:1010E000940C800C450C2C0C410C060C000C440C90
:1010F0005A0C410C930C000C450CAA0C410C940C9E
:10110000000C460C0A0C450C010C000C460C500C53
:10111000450C020C800C460C7E0C450C030C800C1C
:10112000460CBA0C450C110C000C460CDE0C450CA0
:10113000120C800C470C480C450C140C000C470C8E
:10114000C60C450C180C000C480C3C0C450C190C3A
:10115000000C480CD20C450C200C000C480CF40C74
:10116000450C210C100C490C8A0C450C430C000C4E
:10117000490CF40C450C720C000C4A0C640C450C28
:08118000840C000C440C5A0C15
:10180000020C800C4C0C000C040C800C4C0C000CDA
:10181000C00C6E0C010CA00CDD0C000C600CB30CA9
:10182000010C020C200C210C010C010CC00CDE0C74
:10183000000C060C000C000C000C200C210C810C80
:10184000800C940C000CA00CB50C810C400C4A0CC4
:10185000000C600C6B0C810C020C200C210C010C98
:10186000040C200C210C010C800C940C000C400C7E
:101870004A0C000CC00CDE0C000C020C800C4C0C52
:10188000000C010C600CB30C010C060C000C000CDD
:10189000000C800C4C0C800C400C220C010CC00C79
:1018A0006E0C810C200C910C000CA00CDD0C800C3B
:1018B000020C400CAD0C000C020C400CAD0C000CEA
:1018C000A00C520C010C020C400CAD0C000C010CD5
:1018D000A00C520C010C020C000C000C000C400C73
:1018E000AD0C800C020C400CAD0C000C010C000C7B
:1018F000000C000C020CA00C520C010CE00CFF0CB4
:10190000810C020C800C4C0C000C040C000C000C24
:10191000000C400C220C010C200C910C000CE00C73
:10192000FF0C410C080C020C600CB30C010CE00C19
:10193000FF0C810C020C000C8C0C000C080C000C31
:101940008C0C000CA00C9C0C000C400CAD0C000C82
:10195000E00CBD0C000C000CCE0C010CA00CDE0C3D
:10196000010C400CEF0C010CE00C730C010C020C90
:10197000000C0C0C000C100C000C0C0C000C200CBF
:101980001C0C000C400C2C0C000C600C3C0C000CD3
:10199000000C8D0C000C200C9D0C000C400CAD0CB0
:1019A000000C600CBD0C000C000C0E0C010C200C8B
:1019B0001E0C010C400C2E0C010C600C3E0C010C9A
:1019C000000C8F0C010C200C9F0C010C400CAF0C78
:1019D000010C600CB30C010C020C000C8C0C000C04
:1019E000080C000C8C0C000CA00C100C000C400C13
:1019F000210C000CE00C310C000C000C420C010C12
:101A0000A00C520C010C400C630C010CE00C730C8C
:101A1000010C020C000C080C000C0A0CE00CC70CAA
:101A2000000CC00CCF0C000CA00CCF0C000C600CF8
:101A3000CF0C000CE00CCE0C000CE00CCD0C000C1C
:101A4000E00CCB0C000CE00C8F0C000CE00C4F0CED
:101A5000000C000C080C000C020C800C4C0C000C50
:101A6000040C000C000C000CA00CDD0C000CC00CD5
:101A70006E0C010CE00CFF0C010C030CF00C3F0C85
:101A8000000C100CE00C3F0C000CD00C3F0C020CB6
:101A9000B00C3F0C010C700C3F0C030CF00CBE0C96
:101AA000000CF00CBD0C020CF00CBB0C010CF00C8B
:101AB000B70C030CF00C6F0C000CF00C5F0C020C5C
:101AC000F00C7F0C010CF00C7F0C030CF00CFF0CE5
:101AD000000CF00CFF0C020CF00CFF0C010CF00CD5
:101AE000FF0C030C030C000CF80C030C140C000C82
:101AF000000C400C100CC00C010C010CC00C9C0C18
:101B0000030CD00C200C020CD00C0C0C020CE00CC2
:101B1000980C000CE00C4C0C000CF00CC00C000CF1
:101B2000F00C1C0C030CC00C020C000CC00C1E0CA6
:101B3000000CD00CE20C020CD00CCE0C020CE00C11
:101B4000BA0C000CE00C6E0C000CF00CE20C000C5B
:101B5000F00CFE0C030C000CF80C030C400CF80C01
:101B6000030C800C000C000C020C000C0C0C000C84
:101B70000B0CE00C800C010C000C730C000C000C26
:101B8000EC0C010C000CDD0C010C000CBE0C010C6B
:101B9000600C6C0C010C600C5D0C010C600C3E0CBC
:101BA000010CA00CEC0C000CA00CDD0C000CA00C2B
:101BB000BE0C000C020C000C0C0C000C070CE00C12
:101BC000000C010C000C330C000C000C0C0C000C75
:101BD000600C0C0C000C800C0C0C010C000C1D0C8F
:101BE000000C000C2E0C000C020C000C0C0C800CD9
:101BF000000C800C000C090C400C080C000C000CB4
:101C0000040C010C000C0C0C000C400C740C810C2E
:101C1000C00C0B0C810CC00C770C810C400C040C1C
:101C2000810CC00C7B0C810C400C080C810C810CCD
:101C3000000C1B0C800C120C000C000C070C000C90
:101C4000110C000C3E0C150C800C760C2A0C800C30
:101C50007E0C350C800C360C110C800C7E0C2E0C7E
:101C6000800C360C0A0C800C810C000C1B0C800CB8
:101C7000120C000C000C070C000C110C000C2C0CAE
:101C8000150C800C640C2A0C800C6C0C350C800C30
:101C9000240C110C800C6C0C2E0C800C240C0A0CE7
:101CA000800C850C000C1B0C800C120C000C000C22
:101CB000070C000C110C000C3E0C150C800C760C63
:101CC0002A0C800C7E0C350C800C360C110C800C10
:101CD0007E0C2E0C800C360C0A0C800C020C000CB6
:101CE0001E0C800C800C400C000C070C200C120CFD
:101CF000010C000C2D0C000C000C1E0C000C600CD8
:101D0000B30C810C600CB30C010C200C2D0C810C5D
:101D1000200C2D0C010C810C410C770C000C040CD8
:101D2000490C1C0C000C410C140C000C3E0C6B0CF0
:101D3000000C360C630C000C850C410C770C000C6D
:101D4000040C490C1C0C000C410C140C000C3E0C37
:101D50006B0C000C360C630C000CC10C000C360C28
:101D6000800C110C000C000C090C440C240C000C11
:101D7000220C120C000C000C360C000C770C5A0CC8
:101D8000800C7F0C250C800C7F0C5B0C800C770C7E
:101D9000120C800C7F0C6D0C800C770C240C800CCA
:101DA000850C000C360C800C110C000C000C090C7E
:101DB000440C240C000C220C120C000C000C360CF1
:101DC000000C770C5A0C800C7F0C250C800C7F0CBF
:101DD0005B0C800C770C120C800C7F0C6D0C800C53
:101DE000770C240C800C810C000C330C000C040CC0
:101DF000080C080C000C000C000C000C3E0C3B0CFA
:101E0000000C360C330C000C850C000C330C000C51
:101E1000040C080C080C000C000C000C000C3E0C10
:101E20003B0C000C360C330C000C810C000C1B0C12
:101E3000800C020C000C000C090C100C110C000C96
:101E4000240C0A0C000C000C1B0C000C760C2A0C49
:101E5000800C3E0C150C800C7E0C2E0C800C360C6D
:101E60000A0C800C7E0C350C800C360C110C800C8E
:101E7000850C000C1B0C800C020C000C000C090CD7
:101E8000100C110C000C240C0A0C000C000C1B0C88
:101E9000000C760C2A0C800C3E0C150C800C7E0C71
:101EA0002E0C800C360C0A0C800C7E0C350C800C31
:101EB000360C110C800CC10C120C390C000C010CEE
:101EC000000C000C000C850C120C390C000C010CE1
:101ED000000C000C000C030C000C070C000C0D0C8B
:101EE000000C010C020C100C040C000C000C810CFA
:101EF000000C000C040C010C000C410C000C000C3C
:101F0000240C000C000C110C000C000C0C0C000C30
:101F1000000C050C400C080C200C040C000C800C70
:101F2000010C000CA00C000C400C080C400C020C26
:101F3000000C020C800C4C0C000C040C000C000C6F
:101F4000000CC00C6E0C010CA00CDD0C000C600C25
:101F5000B30C010C810C000C1E0C800C000C400C0E
:101F6000000C0C0C300C180C000C260C000C000C97
:101F7000160C000C000C000C500C800C000C440CD7
:101F8000800C000C540C800C000C420C800C000CDB
:101F9000520C800C000C460C800C000C560C800C73
:101FA000000C480C800C000C580C800CC50C000C6C
:101FB0001E0C800C000C400C000C0C0C810C000C56
:101FC000600C800C000C040C000C070C000C480C7E
:101FD000C00C010C000C080C000C580C800C000C00
:101FE000500C800C000C580C800C000C300CC00CF9
:101FF000010C000C050C000C580C800C000C280C7B
:10200000800C850C000C600C800C000C040C000C87
:10201000070C000C480CC00C010C000C080C000C48
:10202000580C800C000C500C800C000C580C800CD0
:10203000000C300CC00C010C000C050C000C580CF2
:10204000800C000C280C800C810C000C1E0C800CE9
:10205000000C400C000C0C0C300C000C000C000CA4
:10206000500C800C000C480C800C000C580C800CA0
:10207000000C440C800C000C540C800C000C420C26
:10208000800C000C520C800C000C4A0C800C000CD4
:102090005A0C800C000C460C800C000C560C800C6A
:1020A000C50C000C1E0C800C000C400C000C0C0C21
:1020B000810C000C1E0C800C000C400C000C100C51
:1020C000060C000C000C000C100C800C000C040C16
:1020D000800C000C140C800C000C020C800C000C0A
:1020E000120C800C000C060C800C000C160C800CE2
:1020F000000C080C800C000C180C800C000C0C0C54
:10210000800C000C1C0C800C000C0A0C800C000CC9
:102110001A0C800C000C0E0C800C000C1E0C800C99
:10212000C50C000C1E0C800C000C400C000C100C9C
:10213000020C000CE00C810C000C080C000C070CCD
:10214000400C4D0C810C800CCD0C800C000C100C44
:10215000400C020C200C700C810C000CB00C800C9C
:10216000000C500C800C200C300C810C810C000CED
:102170003E0C800C010C000C000C0E0C3E0C000CF4
:10218000000C400C000C000C000C610C800C000CCE
:10219000500C800C000C480C800C000C440C800C83
:1021A000000C420C800C000C400C800C560C740C83
:1021B000000C000C5A0C800C000C4C0C800C000C19
:1021C000460C800C000C420C800C000C400C800C67
:1021D000850C000C3E0C800C010C000C000C0E0C4D
:1021E0003E0C000C000C400C000C000C000C610CB0
:1021F000800C000C500C800C000C480C800C000C67
:10220000440C800C000C420C800C000C400C800C28
:10221000560C740C000C000C5A0C800C000C4C0C6E
:10222000800C000C460C800C000C420C800C000C46
:10223000400C800C020CC00C060C800C000C900CA6
:10224000000C070C400C040C000C400CF50C810C2D
:10225000A00CBA0C810C600CFD0C810C400CB40C71
:10226000810CA00CFB0C810C800CB20C810C020CBC
:10227000C00C060C800C000C900C000C070C400CE1
:10228000040C000C400C650C810CA00C2A0C810C79
:10229000600C6D0C810C400C240C810CA00C6B0CA0
:1022A000810C800C220C810C020CC00C060C800CE2
:1022B000000C100C000C090C400C840C000C800C61
:1022C000220C010CC00C060C000CA00CBA0C810CEA
:1022D000400CF50C810CA00CFB0C810C800CB20C9A
:1022E000810C600CFD0C810C400CB40C810C030CB7
:1022F000000C1E0C800C800C400C000C090C100C07
:10230000120C020C000C2D0C000C000C1E0C000C0E
:10231000100C2D0C820C700CB30C830C300C2D0C9B
:10232000830C500CAD0C820C300C330C830C500C15
:10233000B30C820C030C000C0F0C800C100C800CE6
:10234000000C090C000C090C030C800C160C000C82
:10235000000C0F0C000CB00CD60C830CD00CB90C7C
:10236000830CF00CF60C830C900C960C830CF00C88
:10237000F90C830C900C990C830C020C000C1E0CB5
:10238000800C200C000C010C070C000C120C000C33
:10239000600CAD0C810CA00C730C810CE00CED0CEE
:1023A000810C200C2D0C810CE00CF30C810C200C0A
:1023B000330C810C020C800C4C0C000C020C000C39
:1023C000000C000CC00CDE0C000C020C200C210CCC
:1023D000010CA00C6D0C810C020C800C4C0C000C40
:1023E000020C200C210C010CE00CFF0C010C020C67
:1023F000000C000C000C800C4C0C800C030C000C2E
:10240000FC0C830C800C000C000C0B0C000CFF0C63
:10241000030C000CFC0C030C000CFE0C810C100CCB
:10242000FE0C820C200C7E0C830C300CBE0C830C3A
:10243000400CDE0C830C500CEE0C830C600CF60C84
:10244000830C700CFA0C830C000CFA0C030C030CBC
:10245000000C080C000C0E0CF00CF70C030CE00C3C
:10246000FF0C030CD00CFF0C030CB00CFF0C030C86
:10247000700CFF0C030CF00CFE0C030CF00CFD0CAC
:10248000030CF00CFB0C030CF00CEF0C030CF00C29
:10249000DF0C030CF00CBF0C030CF00C7F0C030CD6
:1024A000F00CFF0C020CF00CFF0C010C030C000CE8
:1024B000FC0C030C0B0C000CFF0C030C000CFC0CB4
:1024C000030C000CFE0C010C100CFE0C020C200C7A
:1024D0007E0C030C300CBE0C030C400CDE0C030C09
:1024E000500CEE0C030C600CF60C030C700CFA0C88
:1024F000030CF00CFA0C030C030C000CFC0C030C8A
:102500000B0C000CFF0C030C800CFE0C030C000CDD
:10251000FC0C030C000CFE0C010C100CFE0C020C4D
:10252000200C7E0C030C300CBE0C030C400CDE0C9B
:10253000030C500CEE0C030C600CF60C030C700C2E
:10254000FA0C030C030C800C7F0C000C050C900C97
:102550007F0C020C000C3F0C000CA00C5E0C010C5C
:10256000C00CED0C000CE00CF30C010C810C430CC6
:102570007F0C000C110C000C000C400C100C430CD8
:102580003F0C000C470C5F0C000C130C7F0C000C74
:10259000570C7E0C000C630C770C000C670C6F0C56
:1025A000000C730C7B0C000C770C7D0C000C4A0C9F
:1025B0007F0C000C4D0C7F0C000C5B0C7F0C000C96
:1025C0005F0C7F0C000C6B0C7F0C000C6F0C7F0CF5
:1025D000000C7B0C7F0C000C7F0C7F0C000C850C1E
:1025E000430C7F0C000C110C000C000C400C100C68
:1025F000430C3F0C000C470C5F0C000C130C7F0CC1
:10260000000C570C7E0C000C630C770C000C670C54
:102610006F0C000C730C7B0C000C770C7D0C000C09
:102620004A0C7F0C000C4D0C7F0C000C5B0C7F0CDB
:10263000000C5F0C7F0C000C6B0C7F0C000C6F0C03
:102640007F0C000C7B0C7F0C000C7F0C7F0C000CB3
:10265000030C000C0E0C010C0A0CF00CFF0C010C0E
:10266000000C060C000C000C1E0C000C000C110CD5
:10267000010C800C190C010CC00C150C010CE00CA9
:102680001D0C010CF00C130C010CF00C9B0C010C3C
:10269000F00CD70C010C030C000C0E0C030C0A0CF4
:1026A000000C0F0C030CF00CFE0C010C000C000CC9
:1026B000020C800C080C020CC00C040C020CE00C88
:1026C0000C0C020CF00C020C020CF00C8A0C020C2C
:1026D000F00CC60C020CF00CEE0C020C040C000CFE
:1026E000F80C0F0C0A0C000CFC0C0F0CFC0CFB0C77
:1026F0000F0C000CE00C0F0C000CD20C0F0C000C9B
:10270000B30C0F0C800C730C0F0CC00CF30C0E0CE4
:10271000E00CF30C0D0CF00CF30C0B0CF80CF30CA0
:10272000070C030C000C030C000C110C000C060C25
:10273000000C800C010C000C700CC20C030C400C43
:10274000210C000CB00CE20C030C200C110C000C42
:10275000D00CD20C030C100C310C000CE00CF20C61
:10276000030C000C090C020CF00CCA0C010C000C40
:10277000290C010CF00CEA0C020C000C990C000C5A
:10278000F00C5A0C030C000C790C000CF00CBA0C79
:10279000030C020C000C040C000C100C000C020CBE
:1027A000000CE00CC50C010C000C210C000CE00C22
:1027B000E60C010C800C100C000C600CD70C010C0A
:1027C000400C300C000CA00CF70C010C200C080C79
:1027D000000CC00CCF0C010C000C280C010CE00C00
:1027E000EF0C000C000C980C000CE00C5F0C010CC2
:1027F000000C780C000CE00CBF0C010C030C000C5E
:102800000C0C000C090C100C000C420C080C000CF9
:10281000000C000C000C1E0C000C000C000C010C39
:10282000000C2D0C010C200C000C000CA00C4C0C0E
:10283000000C200C000C010C600C8C0C010C020C28
:10284000100C000C020C100C0C0C820C050CFF0C74
:10285000FF0C000C130CFF0CFF0C020CFF0CFF0C08
:10286000010CFF0CFF0C030CFE0CFF0C000CFD0C0C
:10287000FF0C200CFB0CFF0C100CF70CFF0C300CA9
:10288000EF0CFF0C080CDF0CFF0C280CBF0CFF0C2E
:10289000180C7F0CFF0C380CFF0CFE0C040CFF0C0A
:1028A000FD0C240CFF0CFB0C140CFF0CF70C340C6F
:1028B000FF0CEF0C0C0CFF0CDF0C2C0CFF0CBF0CF6
:1028C0001C0CFF0C7F0C3C0C030C800C7F0C000CD0
:1028D000060CA00C7F0C010C900C730C000C900CDF
:1028E000ED0C000CD00C5E0C000C500CBF0C000C5E
:1028F000800C7F0C020C030C800C4C0C000C050CA3
:10290000000C000C020C400C920C000CA00C6D0C86
:10291000010C300C210C010CD00CDE0C000C030C53
:10292000000CE00C830C200C000C000C0A0CC00CFA
:10293000090C400C200CD00CC10C810C100C3C0C70
:10294000800C100C3C0C830C100C1C0C800C100C1C
:102950001C0C810C100C9C0C800C100C9C0C810C21
:10296000100C980C810C100C8C0C810C030C000CBE
:10297000E00C830C200C000C000C0A0C000C0B0C5F
:10298000400C200C100C630C800C100C7C0C810C87
:10299000100CFC0C800C100CFC0C830C100C1C0C90
:1029A000800C100C1C0C810C100C9C0C800C100C5E
:1029B000980C800C100C8C0C800C020C800CE70C1A
:1029C000810C000C080C000C0E0C200C000C000CF0
:1029D000200C100C800C400C100C800CE00C100C27
:1029E000800CE00C110C800C400C130C800CE00CE3
:1029F000160C800C400C350C800C400C720C800CBA
:102A0000400CD40C800C400CB00C810C400C500CD1
:102A1000810C400C000C000C400C100C800C030CC2
:102A2000000C0C0C800C200C000C000C0B0C400C4F
:102A3000AB0C020C400CAB0C820C100C080C820C82
:102A4000100C080C800C100C040C800C100C080CE2
:102A5000800C100C040C800C100C080C800C100C5A
:102A6000040C800C100C080C800C100C040C800C56
:102A7000030C000C800C800C000C040C000C0D0CE2
:102A8000000C000C020C100C080C820C000C880CC2
:102A9000C20C010C000C070C000C080C820CA00CE2
:102AA000D80C810C000C880C820C000C080C820CD9
:102AB000000C880C820C000C080C820C000C880C9A
:102AC000820C000C080C820C000C880C820C000C90
:102AD000080C820C030CC00C030C800C000C040CC2
:102AE000000C050C000C000C020C400C410C810C7D
:102AF000400CB10C800C800CA20C800C800C4A0C99
:102B0000810C040C100C000C000CD00C030C800C7D
:102B1000200C000C000CE00C030C800C030C200CAF
:102B2000550C820C000C080C000C050C000C000C61
:102B3000000CF00C070C800CC00C020C800C100C6C
:102B4000F00C830C000CA00C810C030C600C360CF8
:102B5000830C000C080C000C070C400C220C010C20
:102B6000500C220C010CB00C250C810CC00C230C59
:102B7000010C500CD20C820C400CE20C010CD00C5D
:102B8000230C010C430C000C7C0C000C000C030CFF
:102B9000600CC60C800C000C000C010C150C700CA9
:102BA000920C020C100CB40C820C400CE40C010CC6
:102BB000400C640C000C000CA00C800C400CA00C11
:102BC000800C200CA00C010CA00CA00C010CA00C83
:102BD000A00C000CA00CA00C010CA00CA10C010C72
:102BE000A00CA10C000CA00CA10C010C200CA10C41
:102BF000010C200CA10C000C400CA10C800C000C52
:102C0000E10C010C000C610C000C400CA50C800CBC
:102C1000000CA50C800C600CA30C800C030C600C49
:102C2000C60C800C000C000C010C150C400C9E0C0A
:102C3000020C200CA60C800C600CE60C010C600C45
:102C4000660C000C000CA00C800C400CA00C800C3E
:102C5000200CA00C010CA00CA00C010CA00CA00CD2
:102C6000000CA00CA00C010CA00CA10C010CA00CE1
:102C7000A10C000CA00CA10C010C200CA10C010C4F
:102C8000200CA10C000C400CA10C800C000CE10CE1
:102C9000010C000C610C000C600CA70C800C200CCB
:102CA000A70C800C400CA70C800C030C600CC60C0D
:102CB000800C000C010C000C100C900CF10C030C9F
:102CC000900CF10C020CF00CD30C020C800CE50CF7
:102CD000800CC00CE50C800CC00CA40C000C800C0B
:102CE000E10C000CC00CE10C800CA00CE10C800C81
:102CF000800C000C400C020CC00CE10C800C800C11
:102D0000E10C800C000C610C000CC00CE50C000CFC
:102D1000800CE50C800CE00CE30C800C030C600CC8
:102D2000C60C800C000C010C000C130C800CF90C70
:102D3000030C800CF90C020CC00CDF0C020CA00C74
:102D4000E60C800CE00CE70C000CE00CA60C000C70
:102D5000800CE00C800CC00CE00C800CA00CE10C92
:102D6000000C200CE10C000CC00CE10C000C400C21
:102D7000E10C000C800CE10C000C000C610C000C50
:102D8000E00CE70C000C600CE70C000CA00CE70C4E
:102D9000000C200CE70C000CC00CE70C000C030C22
:102DA000000CC00C830C000C200C000C110C000C4F
:102DB000000C000C500C990C820C100C480C810C6F
:102DC000300C880C820C100C480C810C100C880CF8
:102DD000800C100C480C800C100C080C800C100C93
:102DE000100C800C100C540C800C100C900C800CEF
:102DF000100C540C810C100CD40C820C100CC40C54
:102E0000820C300CC00C820C100CC40C820C000C18
:102E1000000C000C030C000CE00C830C000C100CDC
:102E2000000C0B0C000C280C000C700C280C820CF5
:102E3000100C280C810C100CA80C800C100C480CE9
:102E4000800C100C280C800C900CA20C820C100C26
:102E5000480C810C100CA80C800C100C480C800C39
:102E6000100C280C800C040C500C550C050C020C9A
:102E7000A80CAA0C020C500C550C050C020C040CEE
:102E8000000C080C540C550C8D0C040C500C550CFB
:102E9000050C020C000C000C080CF80CFF0C0F0CBD
:102EA000020C040C000C000C540C550C850C020C8C
:102EB000800C070C000C060C200C550C010CA00C0F
:102EC0002A0C010C000C780C400C040C800C2A0C11
:102ED000000C000C550C000C800C7F0C400C040CFA
:102EE000040C000C000C010C800C7F0C010C200C5D
:102EF000000C000CA00C7F0C000C040CF80C070C50
:102F0000000C060C500CAD0C020CA80C520C050C5D
:102F1000000CF80C470C040C540CAD0C020CAC0C5F
:102F2000520C050CF80CFF0C470C040C020C000CA6
:102F3000000C080CF80CFF0C0F0C030C000CF80C28
:102F4000030C140C000C000C400C100CC00C010CF9
:102F5000010CC00C9C0C030CD00C200C020CD00CEF
:102F60000C0C020CE00C980C000CE00C4C0C000C4F
:102F7000F00C400C000CF00C1C0C030CC00C020CF0
:102F8000000CC00C0E0C000CD00CE20C020CD00C8F
:102F9000CE0C020CE00CBA0C000CE00C6E0C000C19
:102FA000F00CE20C000CF00CFE0C030C000CF80C06
:102FB000030C400CF80C030C800C000C000C030CF0
:102FC000000C030C000C080C800C010C000C400CD5
:102FD000210C000C200C110C000C100C310C000CFE
:102FE000000C090C020C000C290C010C000C990CB3
:102FF000000C000C790C000C020C000C040C000CF2
:10300000000C070C800C030C800C4C0C000C040C06
:10301000000C820C000CE00C7D0C010C300C200C20
:10302000000CD00CDF0C010C020C000C000C020C8C
:10303000800C4C0C820C030C800C7F0C000C130CCD
:10304000000C000C010C800C800C020C900C800C0D
:10305000030C900C810C020CA00C810C030CA00C36
:10306000830C020CB00C830C030CB00C870C020C0C
:10307000C00C870C030CC00C8F0C020CD00C8F0CF6
:10308000030CD00C9F0C020CE00C9F0C030CE00C0A
:10309000BF0C020CF00CBF0C030CF00CFF0C020C6C
:1030A000700CC00C000C600CC00C010C600CA00C6F
:1030B000000C020C800C610C000C020C400C140C77
:1030C000010C200C8A0C000C040C000C000C000CF1
:1030D000800C610C800C600C9E0C010CE00CFF0C51
:1030E000810C040CC80C940C890C000C080C000C0E
:1030F000040C100C210C020CFC0CF70C8F0C040CB3
:10310000000C800CFC0CF70C8F0C030C800C8C0C4E
:10311000000C040C800C8C0C000C600C620C020C7B
:10312000900C9D0C010CF00CFF0C030C020C000C1D
:10313000060C000C0A0C000C020C000C000C0C0C11
:10314000000C000C1A0C000C000C3C0C000C000CC9
:103150007A0C000C000CFC0C000C000CFA0C010C9E
:10316000200CFC0C010C600CFA0C010C600CFD0C2A
:10317000010C430C900C980C000C040C000C000C7F
:10318000000C430C400C040C800C800C000C000C58
:10319000000C000C200C000C430C000C040C800CE8
:1031A000800C000C000C0A0C000C000C000C100C25
:1031B000240C800C100C240C800C100C240C800CA3
:1031C000100C240C800C100C240C800C100C240C03
:1031D000800C100C240C800C100C240C800C100C97
:1031E000240C800C100C240C800C100C240CC00C33
:1031F000010C000C040C300C200CC00C010C000C59
:10320000030C300C240C800C000C240CC20C010CA0
:10321000000C080C200C200CC20C010C000C0F0C34
:10322000200C240C820C200C240CC20C010C000C71
:10323000200C300C200CC20C010C000C3F0C300C8C
:10324000240C820C030C000CC00C830C000C200C12
:10325000000C020CA00C650C810CA00CB50C820CAF
:10326000040CE00CE30C830C000C100C000C0A0C9A
:10327000000C000C080C040C000C000C040C240CBA
:103280008B0C840C0F0C800C040C640C800C800CD8
:10329000070C880C000C240C8F0C000C240C030C65
:1032A000040C240C0B0C000C2C0C070C020C1C0C3A
:1032B000000C080CFC0CE30C8B0C040CE00CE30C75
:1032C000830C000C100C000C0A0C000C000C880C79
:1032D000040C000C800C040C240C8B0C840C0F0CC4
:1032E000800C040C640C800C800C070C880C000C07
:1032F000240C8F0C000C240C030C040C240C0B0C61
:10330000000C2C0C070C020C1C0C000C080CFC0C08
:10331000E30C8B0C030C000C0C0C000C090C100CB7
:103320000C0C420C080C000C0C0C000C000C120CC9
:10333000000C000C0C0C010C000C210C010C200CDE
:103340000C0C000CA00C400C000C200C0C0C010C04
:10335000600C800C010C020C100C000C020C100C08
:103360000C0C820C040C000C000C0C0C100C000C4F
:10337000020C0A0C000C040C0A0C000C410C0A0C88
:10338000000C440C0A0C800C200C0A0C000C240CC1
:103390000A0C400C600C0A0C000C640C0A0C200C8B
:1033A000100C0A0C000C140C0A0C100C500C0A0C1B
:1033B000000C540C0A0C080C300C0A0C000C340CD9
:1033C0000A0C040C700C0A0C000C740C0A0C060C91
:1033D000000C800C020C000C800C8E0C000C000CFD
:1033E000030C000C000C8F0C000C000C000C000CEB
:1033F000000C8C0C040C000C000C8C0C000C040C4D
:10340000000C100C000C020C8A0C000C000C0A0CB6
:10341000000C410C8A0C000C400C0A0C800C200C97
:103420008A0C000C200C0A0C400C600C8A0C000C5E
:10343000600C0A0C200C100C8A0C000C100C0A0CEE
:10344000100C500C8A0C000C500C0A0C080C300CA0
:103450008A0C000C300C0A0C040C700C8A0C000C4A
:10346000700C0A0C060C000C800C020C000C800C7A
:103470008E0C000C000C030C000C000C8F0C000CCC
:10348000000C000C000C000C8C0C030C400CAD0C60
:10349000000C020C000C000C000CE00CFF0C010CEA
:1034A000040CB00C520C010C500CAD0C800CA00C98
:1034B000520C030C400CAD0C820C030C400CAD0CF8
:1034C000000C020C000C000C000CE00CFF0C010CBA
:1034D000020CB00C520C030C500CAD0C820C040C02
:1034E000C80C940C090C040C000C080C000C000C0B
:1034F000000C000CF80CFF0C0F0CC80C940C090C01
:10350000020C340C630C060CCC0C940C890C040CCF
:10351000C80C940C890C000C080C000C040C000C5A
:10352000000C800C300C630C060CF80CF70C8F0CA4
:10353000C80C940C090C020C340C630C060CCC0C5B
:10354000940C890C030C600CB30C010C040CA00C43
:10355000520C010C300C1E0C030CD00CED0C020CA8
:10356000400CA10C000C040CC80C940C890C000C31
:10357000080C000C040C000C000C800C340C630CC8
:10358000060CF80CF70C8F0CCC0C9C0C090C030CE3
:10359000200C550C820C000C080C000C040C000CC8
:1035A000000C800CD00CA20C010CE00CF70C830C6E
:1035B000300C550C020C030C600C360C830C000C08
:1035C000080C000C040C400C220C810CD00CE30CF9
:1035D000010CA00CD50C820C300C140C020C020C4B
:1035E000800C610C000C040C000C000C000CC00CD6
:1035F000750C010CA00CEB0C000C600C9E0C010C6B
:10360000030C400CBF0C800C900C400C020C060C00
:10361000200C000C010CD00CE10C820C900C520C14
:10362000820CD00CF30C820C900C4C0C820CD00C45
:10363000C00C820C030C400CBF0C800C100C000C56
:10364000020C0B0C200C000C010C500C800C820C9A
:10365000100C210C820C500CA10C820C100C120CC2
:10366000820C500C920C820C100C330C820C500CFF
:10367000B30C820C100C0C0C820C500C8C0C820CB9
:10368000100C000C820C020C800C7F0C800C200CA7
:10369000000C010C070C400C800C000CA00C400C22
:1036A000810C200C210C810C200C120CC10C010C83
:1036B000000C020C200C0C0CC10C010C000C040CB6
:1036C000A00C7F0CC10C010C000C070C200C000C92
:1036D000810C440C000C000C000C000C440C000C81
:1036E000000C000C000C440C000C000C000C000C36
:1036F000030C400CBF0C800C100C000C020C080CCE
:10370000C00CCC0C000C200C000C010C400C800CEC
:10371000800C000C210C800C400CA10C800C000CC7
:10372000120C800C400C920C800C000C330C800CA2
:10373000400CB30C800C000C0C0C800C400C8C0C5E
:10374000800C000C000C800C040C000CF80C070C16
:10375000020CF80C070C000C000CF80C070C040C05
:10376000FC0C070C000C040CF80C870CF80C070C74
:10377000080C000CF80C8F0C040C000CF00C0F0C57
:10378000060C000CF80C0F0C000CF00C0F0CF80CD5
:10379000F70C0F0CF80C0F0C000CF80C070C000CBD
:1037A000000C000C000C020C040C000C000CFC0CB7
:1037B000F70C8F0C040C000CF00C8F0C000C080C98
:1037C000000C040C000CF00C8F0C000CF00C0F0C17
:1037D000F80C070C800C000C000C000C020C040C04
:1037E000000C000CFC0CF70C8F0C430CF00C0F0CB5
:1037F000820C000CA00C000C0D0C000C880C000CB2
:10380000F00C970CC20C010C000CFF0C000C980C77
:10381000800C000C980C820C100C980CC20C010C43
:10382000000C020C100CB80C020C300C980CC20CE2
:10383000010C000C030C300CD80CC20C010C000C59
:10384000020C500C980C800C010C000C030C500C5A
:10385000080C000C000C980C000C100C980CC00C00
:10386000010C000C020CF00C070C420C040C020CB6
:10387000000C000C010CF00C070C830C030C000C6A
:10388000080C800C000C200C000C100CE00C5F0CE1
:10389000010CE00CDF0C010CE00C5F0C010C000CC7
:1038A000180C000C000C180C010C000C180CC10CAE
:1038B000010C000C020C000C100C810C000C180CFC
:1038C000810C000C180CC10C010C000C030C000C3A
:1038D000080C010C000C180C810C000C180C000CCE
:1038E000000C180C810C000C580C810C000C580CAE
:1038F000810C000C100CC10C010C000C020C430CD0
:10390000000C000C800C000C000C000C000C430C94
:10391000000C000C800C000C000C000C000C040CC3
:10392000F80C070C000C040CA80CAA0C020C000CE0
:10393000F80C470C040C540C550C0D0CF80CFF0C37
:10394000470C040C020C000C000C080CF80CFF0CCB
:103950000F0C040CF80C070C000C060C500CAD0CF2
:10396000020CA80C520C050C000CF80C470C040CB3
:10397000540C550C050CAC0CAA0C020CF80CFF0CEA
:10398000470C040C020C000C000C080CF80CFF0C8B
:103990000F0C450C000C000C000C000C450C000C2E
:1039A000000C000C000C030C000CE00C830C200C31
:1039B000000C000C0D0CD00CC10C830CD00C290C8D
:1039C000820C100C280C810C100C080C820C100CB2
:1039D000080C830C100C880C820C100C9C0C820CB4
:1039E000000C9C0C820C000C080C830C000C080CC6
:1039F000800C000C280C830C000C280C820C000C92
:103A0000C80C830C030C000CE00C830C200C000C85
:103A1000000C0D0C500C630C830C500CEB0C820C46
:103A2000100CE80C810C100C080C820C100C080C0B
:103A3000830C100C880C820C100C9C0C820C000C5B
:103A40009C0C820C000C080C830C000C080C800CE5
:103A5000000CE80C830C000CE80C820C000C680CC9
:103A6000830C430C000C000C000C000C440C000CEC
:103A7000000C000C000C440C000C000C000C000CA2
:103A8000440C000C000C000C000C440C000C000C4E
:103A9000000C000C440C000C000C000C000C440C3E
:103AA000000C000C000C000C020C000C340C000C80
:103AB000050C000C340C000C800C480C000C000CA5
:103AC000910C000C000C0A0C010C800CD30C010CA6
:103AD000020C800C610C000C040C800C610C000CBE
:103AE000400C920C000C200C0C0C010C600C9E0C79
:103AF000010C020C200C000C010C060C200C000C1C
:103B0000010C400C100C000C800C200C000C000C64
:103B1000410C000C000C820C000CC00CF30C000CCF
:103B2000820C200C820C000C040CC00C000C000C4D
:103B3000A00C830C000C000C010C000C600C820C1F
:103B4000000C020C800C610C000C040C800C610C4D
:103B5000000CC00CF30C000CA00C6D0C010C600CE4
:103B60009E0C010C020C200C000C010C060C200C0D
:103B7000000C010C600C100C010CA00C200C010CB2
:103B8000200C410C010C200C820C010CC00CF30C1D
:103B9000000C020C600C800C810C800C400C000CA2
:103BA000050C200C0C0C010C400CA10C000C600C42
:103BB000AD0C010C400C800C800C200C120C810C04
:103BC000030CE00CF10C800C100C080C000C060C23
:103BD000000C020C010C000C850C820C800C400CBB
:103BE000800C400CA50C820CA00C500C800C000C1E
:103BF000060C030C020CC00C300C000C020C000C68
:103C0000860C010CE00CFF0C010C020C000C000CEB
:103C1000000CC00C300C800C030CF00C7F0C800CE2
:103C2000000C000C010C110C400C400C020C200C80
:103C3000400C800C800C400C800C000C440C800C60
:103C4000000C500C800C100C000C800C000C010CB3
:103C5000800C000C020C800C000C080C800C000C7A
:103C6000200C800C400C400C010C000C800C400C13
:103C7000020C200CC00C810C800CC00C810C000CC0
:103C8000C40C810C000CD00C810C400CC00C030C3B
:103C9000830C800CA30C800C000C000C010C170C86
:103CA000800CA30C820C800CA20C800C000CA20CCB
:103CB000800C000CA00C800C000C800C800C000C04
:103CC000000C800C000C010C800C800C010C800C92
:103CD000800C030C800C800C230C800C800CA30C3B
:103CE000800C800CA20C800C000CA20C800C000C30
:103CF000A00C800C000C800C800C000C000C800CC4
:103D0000000C490C800C800C5B0C000C800C5B0CD4
:103D1000800C800C230C800C800CA30C800C800C7D
:103D2000A20C800C000CA20C800C030C000CF00CFC
:103D3000000C0E0C000C000C000CF00C070C020C1C
:103D4000F00CFF0C020CF00CF70C030C000C080C30
:103D5000010C000C880C030C100C880C010C200CBE
:103D6000480C010C400C480C010C800C280C010C78
:103D7000000C290C010C000C1A0C010C000C1C0C82
:103D8000010CF00CFF0C030C030CF00CCF0C830C9B
:103D9000000C100C000C0F0C000C200C000C000C84
:103DA000180C800C000C140CC00C010C000C070C3F
:103DB000000C110CC00C010C000C080C800C100C39
:103DC000C00C010C000C100C000C120CC00C010CEF
:103DD000000C200C000C900CC00C010C000C400CD2
:103DE000000C500CC00C010C000C800C000C100CD2
:103DF000C10C010C010C000C000C100CC20C010CCD
:103E0000020C000C100C100CC00C010C040C000C6B
:103E1000200C100CC00C010C080C000C400C100CF9
:103E2000C00C010C100C000CF00CDF0CC30C010CCE
:103E30001F0CFF0C000C100C800C030C600C400CD1
:103E4000800C000C100C000C070C000C080C400C33
:103E5000200CF00C0A0C410C200C000CCD0C420C78
:103E6000200CF00CCF0C430C200C400C400CC00C70
:103E7000010C000C060C000C200CC00C010C000CFA
:103E8000020C200C400CC00C010C000C050C030CA7
:103E9000F00C750C800C000C000C010C0B0C200CB1
:103EA000400C020C100C400C800C400C400C800CA0
:103EB000000C440C800C000C200C800C800C000CBE
:103EC000800C000C010C800C000C100C800C200CE1
:103ED000400C800C200CC00C010C100C400C010C90
:103EE000020C000C340C000C050C000C340C000C03
:103EF000A00C340C010C400CB50C000C000C7E0C1A
:103F0000010CE00CCB0C010C020C800CD70C800CCB
:103F1000200C000C000C0E0C400C000C000C200CB3
:103F2000800C800C200C400C800C200CC00C800CF1
:103F3000200C100C800C200C900C800C200C500CD1
:103F4000800C200CD00C800C200C040C800C200C5D
:103F5000020CC00C010C000C080C200C010CC00C55
:103F6000010C000C100CA00C000CC00C010C000C7F
:103F7000200CA00CD70CC00C010C000C3F0C200C2A
:103F8000000C800C020C000C340C000C050C000C16
:103F9000340C000CA00C000C010C400C810C000C2B
:103FA000000C4A0C000CE00CCB0C010C030C300C88
:103FB000000C830C400C800C000C090C100C0C0C39
:103FC000020CA00C400C010CB00C4C0C030C200C8F
:103FD000210C810C200C000C810C100C120C820C9A
:103FE000200C330C810C100C330C820C100C000CC8
:103FF000820C030CF00C0F0C030C100C400C000C8A
:10400000000C000C100C010C200C800C000C000C9F
:10401000900C020C100C400C000C000C520C000C0C
:10402000000CC40C000C800CD00C000C000C280CF4
:10403000000C000C310C000C000CA00C000C000C4F
:10404000B00C000C000C600C000C000C700C000C90
:10405000000CE00C000C000CF00C000C030C200C0D
:10406000260C810C000C000C020C170C100C140C0C
:10407000000C000C160C800C000C340C800C000C96
:10408000360C800C000C140C810C000C160C810CEE
:10409000000C340C810C000C360C810C200C140C20
:1040A000800C200C120C800C200C040C800C000CDA
:1040B000260C810C000C240C810C000C060C810CCD
:1040C000000C040C810C000C260C800C000C240C41
:1040D000800C000C060C800C000C000C800C000CFA
:1040E000050C800C200C060C800C100CE40C010C50
:1040F000000CF60C810C020C800C610C000C040C02
:10410000000C000C000CC00CF30C000CA00C6D0C8F
:10411000010C600C9E0C010C030CF00CCF0C830CFA
:10412000000C100C000C0F0C000C200C000C000CF0
:10413000180C800C000C140C800C000C120CC00C21
:10414000010C000C020C000C110CC00C010C000C3A
:10415000040C400C100CC00C010C000C080C200CC2
:10416000100CC00C010C000C100C800C100CC00CBE
:10417000010C000C200C000C900CC00C010C000C6D
:10418000400C000C500CC00C010C000C800C000CFE
:10419000100CC10C010C010C000C000C100CC20C1A
:1041A000010C020C000C100C100CC00C010C040CC7
:1041B000000CF00CDF0CC30C010C070CFF0C000C06
:1041C000100C800C030C300C180C000C050CF00CBF
:1041D0007F0C030C400C250C020C000C010C000C95
:1041E000B00C5B0C010C300C190C000C020C000C18
:1041F000000C000C300C180C800C030C100C980CEC
:10420000000C050C000C010C000C400C250C020CE1
:10421000C00C670C030C900CDB0C010CD00CFF0CD9
:10422000030C020C000C000C000C100C980C800C01
:10423000C10C600C000C800C000C400C000C000C3D
:10424000000C000C000C830CA00C520C020C020C95
:10425000A00C520C020C400C2D0C010C850CA00C77
:10426000520C020C020CA00C520C020C400C2D0C37
:10427000010C030C400C000C000C120CB00C410C97
:10428000030CB00CE10C020CB00CD10C010CB00C06
:10429000B10C030CA00CC90C030CB00CE80C030C03
:1042A000900CD90C030C300CF90C030C400C800C56
:1042B000000C400C200C010C400C100C020C400CAB
:1042C000700C000C500C080C000C400C290C000C5D
:1042D000600C180C000CC00C380C000C000C820C8C
:1042E000000C800C3A0C000C030C400C800C000CF1
:1042F0000A0CA00C210C030CB00C700C020C900CDE
:10430000690C010C300C590C030C500CC00C000C47
:10431000400C910C010C600C880C020CC00CB80C09
:10432000000C100C420C000C800C3A0C000C030C1E
:10433000800C000C030C0A0C500C800C000C500C70
:10434000A00C010C500C900C020C500CB00C030C87
:10435000D00C880C000CD00CA80C010CD00C980CC4
:10436000020CD00CB80C030C200C430C000C500CAD
:10437000BA0C000C030CF00C870C830C000C200C06
:10438000000C0D0C000C400C000C000C240CC00C9C
:10439000010C000C080C000C210CC00C010C000CD2
:1043A000080C800C200CC00C010C000C100C000C34
:1043B000220CC00C010C000C200C000C200CC10CB9
:1043C000010C000C400C000CA00CC00C010C000CEB
:1043D000800C000C200CC20C010C010C000C100C09
:1043E000200CC00C010C040C000C200C200CC00C88
:1043F000010C080C000C400C200CC00C010C100C23
:10440000000CF00CA70CC30C010C1F0CFF0C000CD3
:10441000200C800C020C200C000C010C0A0CE00C8F
:10442000F30C000C800CF30C010C400CF30C010C91
:10443000C00CF20C010CC00CF10C010CC00CE30C14
:10444000010CC00CD30C010CC00CB30C010CC00C43
:10445000730C010C000C000C010C020C400CAD0C98
:10446000000C020C400CAD0C000CA00C520C010C0A
:10447000030CC00C030C800C000C040C000C050C8D
:10448000000C000C020C400C410C810C400CA90CDF
:10449000800C800CA20C800C800C520C810C040C43
:1044A000100CA00C000CD00CA30C800C200C400CA9
:1044B000010CE00C430C810C020C200C000C010CD4
:1044C0000A0C000C000C010C600C000C000CA00C81
:1044D000000C000C200C010C000C200C020C000C39
:1044E000200C100C000C200C200C000C200C400C9C
:1044F000000C200C800C000CE00CF30C000C020CE7
:10450000800C000C000C060C800C400C000CA00C65
:10451000CA0C000CC00C540C010C600CDE0C010C1D
:10452000000C600C000C000C000C000C030C800C48
:10453000FF0C810C400C000C000C100C100C000C3B
:10454000820CB00C000C820C100C010C820CB00C14
:10455000020C820C100C050C820CB00C020C830CAB
:10456000B00C850C820C100C430C830C500CAE0C60
:10457000020C300CBE0C020CF00C540C030CA00C02
:10458000440C030CE00C940C030CA00C9C0C030CCE
:10459000E00C940C030CA00C940C030C020C000C0B
:1045A000180C000C800CFF0C810C030C600CC60C6A
:1045B000800C000C010C000C0D0C800CF90C030C91
:1045C000C00CDF0C020CA00CE60C800CE00CA60C5E
:1045D000800C800CE00C800CC00CE00C800CA00C5B
:1045E000E10C000C800C000C400C020C400CE10CA7
:1045F000800C000C610C800C600CE70C800C200C13
:10460000E70C800CC00CE70C000C030C000CC00C79
:10461000830C000C200C000C090C000C000C000C8E
:10462000100C540C800C100C900C800C300C840C72
:10463000800C300C480C820C100C080C810C300CD7
:10464000040C810C500C990C820C900C5A0C810CAF
:10465000030C000C900C030C060C000C900C010CCD
:10466000100CB10C020C200CD20C020C400CB40C3F
:10467000020C800CD80C020CF00C6F0C020C030C1A
:10468000200C2D0C010C040C200C2D0C010C500CDA
:10469000920C020C000C400C000C500CD20C020CC2
:1046A000040C800C000C000CA00C6D0C810CD00CC8
:1046B000920C020CF00CFF0C830C030C400CAD0CA4
:1046C000000C020C000C000C000CE00CFF0C010CA8
:1046D000020CB00C520C030C500CAD0C820C030CF1
:1046E000000CF80C030C100C000CF80C030C400C24
:1046F000000C000CC00CF80C020CC00C640C000C7C
:10470000D00CD80C010CD00CF40C010CE00C600C9B
:10471000030CE00CB40C030CF00C380C030CF00C84
:10472000E40C000CC00CFA0C030CC00CE60C030CDF
:10473000C00CE10C030CD00C020C000CD00C060CCD
:10474000000CE00C020C000C030C000C000C010C23
:10475000110C100C000C010CE00C0F0C000C200CC8
:10476000200C010CD00C2F0C000C400C400C010C48
:10477000B00C4F0C000C800C600C010C700C6F0C1A
:10478000000C000C810C010CF00C8E0C000C000CC9
:10479000A20C010CF00CAD0C000C000CC40C010CB4
:1047A000F00CCB0C000C000CE80C010CF00CE70C2E
:1047B000000C000CF80C000C020C100C000C020C8D
:1047C000000C100C830C050CF80CFF0C070C120CE1
:1047D000010C040C000C030C010C000C050C020C69
:1047E000000C870C000C000C410C000C080C230C76
:1047F000000C080C150C000C080C0F0C000C080C1D
:10480000010C000C110C030C800C100C050C000C9E
:10481000140C070C000C120C010C100C180C030CDF
:10482000080C180C050C400C180C000C400C000C6B
:10483000070C200C180C010C000C200C030CC00CF5
:10484000E30C810C100C080C000C160C000C040C72
:10485000020C600C300C800CA00C500C800CE00C96
:10486000700C800C200C910C800C600CB10C800C36
:10487000A00CD10C800CE00CF10C800C200C120C64
:10488000810C600C320C810C200C100C800C200C64
:10489000100C400C020C600C300C800CA00C500C66
:1048A000800CE00C700C800C200C910C800C600CC7
:1048B000B10C800CA00CD10C800CE00CF10C800C25
:1048C000200C120C810C400C220C010C000C040C6E
:1048D000020C030C000CF00C000C040C300C010C4E
:1048E000020C300CA30C010C300C5B0C000C300CD7
:1048F000990C030C030CC00CE30C810C100C080C7D
:10490000000C160C000C040C020C600C300C800C1B
:10491000A00C500C800CE00C700C800C200C910C46
:10492000800C600CB10C800CA00CD10C800CE00C45
:10493000F10C800C200C120C810C600C320C810CE0
:10494000A00C520C810C200C100C400C020CE00C42
:10495000720C810C200C930C810C600CB30C810C3C
:10496000A00CD30C810CE00CF30C810C200C100C6F
:10497000800C600C300C800CA00C500C800CE00CF7
:10498000700C800C000C040C020C030C100CF00CCE
:10499000830C000C020C000C0C0C200C000C000C06
:1049A000000C120CC00C400C000C080C000C220C6B
:1049B000C00C400C000C080C000C420CC00C400C4D
:1049C000000C100C000C820CC00C800C000C200C95
:1049D000000C020CC10C800C000C400C000C020CF2
:1049E000C20C800C000C800C100C020CC00C800C53
:1049F000010C000C030C000CF80C030C110C000C47
:104A0000040C000C100CF80C020C100C310C000CF7
:104A1000500CD80C010C500C790C010C300C300CE3
:104A2000030C300C690C030C700CE80C030C700CBC
:104A3000390C000C900CF80C030C900C790C030C46
:104A4000D00C000C000CD00C010C000CB00C000CB5
:104A5000000CB00C010C000CF00C000C000CF00C65
:104A6000010C000C030C500CA90C000C040C500C95
:104A7000A90C000CA00C560C030C500CAA0C010C39
:064A8000A80CD40C020C8E
:020000040030CA
:0300010022090EC3
:02000500008079
:060008000FC00FE00F40E5
:00000001FF
